:020000020000FC
:100000000EC00DC00CC00BC00AC009C008C007C09C
:1000100006C005C022C003C002C001C000C002E08B
:100020001FE50EBF1DBF0024112422244424662492
:100030006394AA24992433274427479A04E008BBF1
:1000400003E007BB02E00ABD09EF09BD00E109BFFB
:1000500002E003BF78948895FECF44FF04C008B344
:1000600013E0012708BB03940AEF0016B1F4002443
:1000700013940CE3101689F41124239405E0201640
:1000800061F4222443940CE0401639F44424639430
:100090000DE0601611F401E0602E30FD0CC031FD62
:1000A00013C032FD22C033FD25C034FD39C035FDFB
:1000B0003FC031E04EC0989400FE8A9421F4330F83
:1000C000762C542C322C45C0772021F4330F0AEFC4
:1000D000802E3FC0002D002311F4C09AC1980D3727
:1000E00019F4C098C1987A9434C08A9491F5330F6A
:1000F000842C2FC0552049F4377F992011F03061AE
:1001000001C031600AEF802E24C0002D002311F4BD
:10011000C19AC0980D3719F4C198C0985A9419C063
:100120008A94B9F4330F092D0F3F09F09A9411C046
:10013000332021F431E00AEF802E0BC0002D002384
:1001400011F44061C19A0D3721F44F7EC198C098D7
:100150003A94002D037021F443FF03C0477F4460AD
:100160003DC008B314E018BB00000000B29B24C0DF
:1001700008BB41FF15C040FF06C0992011F099242B
:1001800019C09A9417C01124239405E0201630F06A
:10019000222443941CE0411608F04424902E0AC007
:1001A00040FF08C063940DE0601610F0662463946D
:1001B00005E0902E487F12C0C09A00000000B29B5C
:1001C0004260C098C19A00000000B29B416008BB29
:0E01D00041FD486040FD486042FD477F1895A4
:00000001FF
